:1000000083161F308500F0308600640007308100C1
:10001000831264008519092886016400051A0C28DA
:100020003620051A0C280130860020200230860078
:1000300020200430860020200830860020200C2854
:100040006400851920288101910192016400811FBB
:1000500026288101851D3128920A1208013C0319C6
:100060003628910A1108963C031D2628810191012A
:100070006400811F38288101910A11080A3C031D80
:040080003828080014
:02400E00F53F7C
:00000001FF
